:100000000C942A000C9447000C9447000C94470071
:100010000C9447000C9447000C9447000C94470044
:100020000C9447000C94A9000C9447000C944700D2
:100030000C9447000C9447000C9447000C94470024
:100040000C9447000C9447000C9447000C94470014
:100050000C94470011241FBECFE5D4E0DEBFCDBF16
:1000600010E0A0E6B0E0E0EBF4E002C005900D92F5
:10007000A036B107D9F710E0A0E6B0E001C01D92AC
:10008000A236B107E1F70E94DB000C9456020C94F3
:100090000000B89AC09A8FE39CE90197F1F700C07D
:1000A0000000C0988AEC90E090936100809360001B
:1000B0008FEF96E1A1E181509040A040E1F700C0B0
:1000C000000010926100109260008FEF96E1A1E1B4
:1000D00081509040A040E1F700C000000895CF9308
:1000E000DF9300D0CDB7DEB719821A82CE01019618
:1000F00062E00E94E9018981873329F48A8183368D
:1001000011F40E9449000F900F90DF91CF91089554
:10011000CF93DF930F92CDB7DEB781E08983CE0115
:10012000019661E00E94A1018FEF90E7A2E081506B
:100130009040A040E1F700C000000F90DF91CF9108
:10014000089585E083BF88E582BF1CBE81E089BF3A
:1001500008951F920F920FB60F9211242F933F9381
:100160008F939F9388E582BFB99AC19A8FEA94E0F2
:100170000197F1F700C0000080916000909161004C
:100180001816190674F480E090E025E12A95F1F73D
:100190000000019620916000309161008217930762
:1001A000A4F3C1989F918F913F912F910F900FBE13
:1001B0000F901F9018950E940D0180E296E00E941A
:1001C000550181E060E047E00E94370180E895E258
:1001D0000E94650180E066E00E948C010E94A100FF
:1001E00078940E946F00FDCF939840E120E030E0CA
:1001F000992314F4959A01C09598220F331F86997C
:100200002160949A880F991F00C000009498415073
:1002100079F7939A822F932F089588E381BB88E022
:1002200082BB8FEF90E7A2E081509040A040E1F7C1
:1002300000C0000080EE90EC0E94F40087ED90E892
:100240000E94F4008BEA92EC0E94F40081E89AECA0
:100250000E94F40080E090EE0E94F40080E098ECB0
:100260000E94F40087EF94EC0E94F400089590E05F
:10027000880F991F82959295907F9827807F982765
:10028000907050E047705070842B952B946970E00B
:1002900063707070660F771F660F771F660F771F8A
:1002A000862B972B0E94F40008958036910538F034
:1002B0002FE08034920728F08FE39FE002C080E6B1
:1002C00090E0906A0E94F400089522E08739920736
:1002D00010F125E18831920780F49C0140E050E064
:1002E00060E678EA80E090E00E943B02C901019755
:1002F0008068966C0E94F40008959C0140E050E0F4
:100300006CEF72E485E090E00E941902C901019748
:10031000966C0E94F400089590E087709070986940
:1003200070E062957295707F7627607F7627707097
:10033000862B972B0E94F40008959398869BFECFFE
:1003400008950F931F93CF93DF938C01C62F88E3FB
:1003500092E80E94F4000E949D018AEA98EB0E94B4
:10036000F4000E949D018AEA98EB0E94F4000E942A
:100370009D018AEA98EB0E94F4000E949D018DE2A3
:1003800098EB0E94F4000E949D0184ED98EB0E947E
:10039000F400CC2399F0C8010196C1509C012C0FA8
:1003A000311DE9010E949D01F80181918F0190E0CA
:1003B000986B0E94F4000C171D07A1F70E949D0185
:1003C00088E092E80E94F400DF91CF911F910F9195
:1003D00008950F931F93CF93DF938C01D62F88EC52
:1003E00092E80E94F40081E89AEC0E94F40083E80D
:1003F0009AEC0E94F400DD2399F0C8010196D150D7
:100400009C012D0F311DE9010E949D0180E090EBC0
:100410000E94F400F80181938F01EC17FD07A1F70A
:1004200088E092E80E94F400DF91CF911F910F9134
:100430000895A1E21A2EAA1BBB1BFD010DC0AA1F25
:10044000BB1FEE1FFF1FA217B307E407F50720F03D
:10045000A21BB30BE40BF50B661F771F881F991FB8
:100460001A9469F760957095809590959B01AC0101
:10047000BD01CF01089597FB092E05260ED057FD2B
:1004800004D0D7DF0AD0001C38F450954095309541
:1004900021953F4F4F4F5F4F0895F6F79095809508
:1004A000709561957F4F8F4F9F4F0895F894FFCFC0
:00000001FF
